:020000040000FA
:020000000428D2
:08000800FF30A200FF30A3004D
:100010000130A400FF30A5000130A6000130A70088
:10002000A010C3222A087F39C822A9222210BC228C
:100030002217B6222211BA22A211B9222212B82204
:10004000A212B722A214BB22A217B5222310B422F7
:10005000A310B3222311B222A311B1222312B02282
:10006000A312AF222313AE22A313AD22FE30A800A9
:10007000A7212508AD002608AE002708AF002408F8
:10008000AF21A60A851C4528EC20051B48285128CD
:100090002508AD002608AE002708AF002408AF21D0
:1000A0004528A80B3828FE30A800A7212508AD0058
:1000B0002608AE002708AF002408AF210130250232
:1000C000A500851C6428EC20051B672870282508DE
:1000D000AD002608AE002708AF002408AF21642831
:1000E000A80B5528FE30A800A7212508AD0026083A
:1000F000AE002708AF002408AF21A70A851C81287D
:10010000EC20051B84288D282508AD002608AE00AC
:100110002708AF002408AF218128A80B7428FE30DF
:10012000A800A7212508AD002608AE002708AF00CB
:100130002408AF2101302602A600851CA028EC204F
:10014000051BA328AC282508AD002608AE0027080B
:10015000AF002408AF21A028A80B9128FE30A800EA
:10016000A7212508AD002608AE002708AF00240807
:10017000AF21A50A851CBD28EC20051BC028C92875
:100180002508AD002608AE002708AF002408AF21DF
:10019000BD28A80BB028FE30A800A7212508AD0077
:1001A0002608AE002708AF002408AF21013027023F
:1001B000A700851CDC28EC20051BDF28E828250883
:1001C000AD002608AE002708AF002408AF21DC28C8
:1001D000A80BCD283628EB28FF30A9000130AA0053
:1001E0000130AB00FE30AC00A7218518F828A62905
:1001F0002908AD002A08AE002B08AF002408AF2163
:10020000AC0BF428051B05290E292908AD002A0886
:10021000AE002B08AF002408AF210229FF30AA004E
:10022000FE30AC00A72185181629A6292908AD00A3
:100230002A08AE002B08AF002408AF21AC0B12290E
:10024000051B23292C292908AD002A08AE002B08FC
:10025000AF002408AF2120290130A900FE30AC00F6
:10026000A72185183429A6292908AD002A08AE003F
:100270002B08AF002408AF21AC0B3029051B412906
:100280004A292908AD002A08AE002B08AF0024082F
:10029000AF213E29FF30AB00FE30AC00A72185180E
:1002A0005229A6292908AD002A08AE002B08AF0064
:1002B0002408AF21AC0B4E29051B5F2968292908AA
:1002C000AD002A08AE002B08AF002408AF215C293E
:1002D0000130AA00FE30AC00A72185187029A6299C
:1002E0002908AD002A08AE002B08AF002408AF2172
:1002F000AC0B6C29051B7D2986292908AD002A082D
:10030000AE002B08AF002408AF217A29FF30A900E6
:10031000FE30AC00A72185188E29A6292908AD003A
:100320002A08AE002B08AF002408AF21AC0B8A29A5
:10033000051B9B29A4292908AD002A08AE002B081B
:10034000AF002408AF2198290130AB000800851FB9
:10035000AC291E30A400AE290130A4000800B00072
:100360002011A0112012A0122013A0132D082E027C
:10037000031DD3292D082F02031DD3292F08023C6A
:100380000318C92902302F02AF0001302E02AE003F
:10039000D2292F08023C031CD2292F08013EAE00AF
:1003A0000230AD07082A2D082E02031DE5292D086D
:1003B000023C0318DF2901302E02AE00E4292D088B
:1003C000023C031CE429AD0A082A2D082F02031D54
:1003D000F7292D08023C0318F12901302F02AF0044
:1003E000F6292D08023C031CF629AD0A082A2F081D
:1003F0002E02031D082A2F08023C0318032A01308D
:100400002E02AE00082A2F08023C031C082AAE0A5E
:100410002D082E0203183B2A2E082F020318192A32
:100420002F08B1002E08B2002D08B30020162017A7
:100430003A2A2F082E0203182A2A2F082D02031801
:100440002A2A2E08B1002D08B2002F08B300A015EB
:10045000A0163A2A2F082E0203183A2A2D082F0236
:1004600003183A2A2E08B1002F08B2002D08B30055
:10047000A015A0176D2A2E082D0203186D2A2F082B
:100480002E0203184C2A2D08B1002E08B2002F08A6
:10049000B300201520176D2A2E082F0203185D2A9D
:1004A0002F082D0203185D2A2D08B1002F08B20075
:1004B0002E08B3002015A0176D2A2E082F0203184E
:1004C0006D2A2D082F0203186D2A2F08B1002D0860
:1004D000B2002E08B3002016A0163308B40032086C
:1004E0003302B30031083202B20083168330620057
:1004F00083123108FF3CB5003208FF3CB6003308D8
:10050000FF3CB7000B11350881000617861606164A
:10051000A42220190613A0198612201A06123608E2
:100520008100A422A01A0613201B8612A01B06120B
:1005300037088100A42206138612061234088100AF
:10054000A422B00B822AA82A0B1DA42A0B11080092
:100550000800CC2207309F000800BD2ABD2ABD2A12
:10056000BD2ABD2ABD2ABD2ABD2AC02AC02AC02A4A
:10057000C02AC02AC02AC02AC02A23086600080050
:100580002208650008000108AB002B08AA0008003B
:0E059000A80028086200080083120313080068
:02400E00623F0F
:00000001FF
